:1000000000308A0004280000FF238316900000308F
:100010008A00532A0A108A100A1182073F340634D4
:100020005B344F3466346D347D3407347F346F3441
:1000300077347C3439345E34793471342730840039
:100040000008031932280130A100A001A00B2628C6
:10005000A10B25284A30A000A00B2C28000000008E
:10006000800B232800342030B900B501B601B70158
:10007000B8013008A3002F08A2002E08A1002D0807
:10008000A0000310201C52283108B50732080318BD
:10009000320FB60733080318330FB70734080318B5
:1000A000340FB807B80CB70CB60CB50CA30CA20CE7
:1000B000A10CA00CB90B41280034A001A101A201A0
:1000C000A301B901BA01BB01BC01380837043604E9
:1000D000350403199B282030BD000310B10DB20D6B
:1000E000B30DB40DB90DBA0DBB0DBC0D38083C02F3
:1000F000031D842837083B02031D842836083A0272
:10010000031D842835083902031C95283508B902D7
:100110003608031C360FBA023708031C370FBB0220
:100120003808031C380FBC020314A00DA10DA20D4A
:10013000A30DBD0B6D280000393084000034B101DF
:100140003108073C031CC328B01FAB288316851257
:1001500083128516AF288316851283128512031029
:10016000B00D0330A000A00BB32883160511831235
:1001700005150330A000A00BBB28831605118312C0
:100180000511B10AA0280034831605118312051148
:1001900083160512831205120330A000A00BCE288F
:1001A0002D08B0009F202E08B0009F202F08B0001F
:1001B0009F200330A000A00BDB28831605128312BA
:1001C00005160330A000A00BE32883160512831246
:1001D000051200340030A1001F08C33921049F001C
:1001E0000330A000A00BF2289F149F18F528831657
:1001F0001E088312A9001E08AA00AB01AC012C083E
:10020000B0002B08AF002A08AE002908AD00B401E9
:10021000B3010130B200F430B10033202308B00044
:100220002208AF002108AE002008AD002308B4006A
:100230002208B3002108B2002008B100B801B701BC
:100240000330B600FF30B5005D202308AC00220863
:10025000AB002108AA002008A9002C08B4002B0834
:10026000B3002A08B2002908B100B801B701B601ED
:100270000A30B5005D200008A8002C08B4002B0847
:10028000B3002A08B2002908B100B801B701B601CD
:100290000A30B5005D202308AC002208AB0021081D
:1002A000AA002008A9002C08B4002B08B3002A08D3
:1002B000B2002908B100B801B701B6010A30B50093
:1002C0005D200008A7002C08B4002B08B3002A0802
:1002D000B2002908B100B801B701B6010A30B50073
:1002E0005D202308AC002208AB002108AA002008EA
:1002F000A9002C08B4002B08B3002A08B200290872
:10030000B100B801B701B6010A30B5005D200008A0
:10031000A600A6080319902926080A20A100A60015
:1003200027080A208038A70028080A20A100A80072
:100330002608AD002708AE002808AF00C420872A91
:100340000430A1001F08C33921049F000330A0001E
:10035000A00BA8299F149F18AB2983161E0883128F
:10036000A9001E08AA00AB01AC012C08B0002B08A4
:10037000AF002A08AE002908AD00B401B301033074
:10038000B200E730B10033202308B0002208AF00EC
:100390002108AE002008AD002308B4002208B300F5
:1003A0002108B2002008B100B801B7010330B6003F
:1003B000FF30B5005D202308AC002208AB00210807
:1003C000AA002008A9002C08B4002B08B3002A08B2
:1003D000B2002908B100B801B701B6010A30B50072
:1003E0005D200008A8002C08B4002B08B3002A08E0
:1003F000B2002908B100B801B701B6010A30B50052
:100400005D202308AC002208AB002108AA002008C8
:10041000A9002C08B4002B08B3002A08B200290850
:10042000B100B801B701B6010A30B5005D2000087F
:10043000A7002C08B4002B08B3002A08B200290832
:10044000B100B801B701B6010A30B5005D2023083C
:10045000AC002208AB002108AA002008A9002C0843
:10046000B4002B08B3002A08B2002908B100B80173
:10047000B701B6010A30B5005D200008A6002608C5
:100480000A208038A60027080A20A100A700280813
:100490000A20A100A8002608AD002708AE00280801
:1004A000AF00C420892A84011F30830583161F08EA
:1004B000F03907389F00073083129F00FA30A700F9
:1004C0001E20831685118312851583161F08F039A7
:1004D00001389F001F08F03902389F001F08F039CB
:1004E0009F001F080F3930389F0083121F080C39F6
:1004F00081389F00FA30A7001E2083168515003032
:10050000831285190130013C031D882AEA28892AB3
:10051000A0290230A600FA30A7001E20A60B8B2AC5
:040520007D2A6300CD
:02400E008431FB
:00000001FF
